:020000001028C6
:1000200000008312850186019201930190018C01E9
:10003000910160308D001F3083168101811785008A
:1000400083127F30831686008312051C2C289201B0
:10005000851D4A2893012528920A921D372892016E
:10006000800110308D0760300D0703196620861758
:10007000A53091000D088C008C0F3C28910F3A2878
:100080008613A53091000D088C008C0F4528910F28
:1000900043282528930A931D53289301800110308B
:1000A0008D0203198D078617003090000D088C0013
:1000B0008C0F5828900F56288613A53091000D08F4
:1000C0008C008C0F6128910F5F282528800110304B
:0400D0008D02080095
:00000001FF
